:020000020000FC
:100000000C944600FFFFFFFFFFFFFFFFFFFFFFFF16
:10001000FFFFFFFFFFFFFFFFFFFFFFFFFFFFFFFFF0
:10002000FFFFFFFFFFFFFFFFFFFFFFFFFFFFFFFFE0
:10003000FFFFFFFFFFFFFFFFFFFFFFFFFFFFFFFFD0
:10004000FFFFFFFFFFFFFFFFFFFFFFFFFFFFFFFFC0
:10005000FFFFFFFFFFFFFFFFFFFFFFFFFFFFFFFFB0
:10006000FFFFFFFFFFFFFFFFFFFFFFFFFFFFFFFFA0
:10007000FFFFFFFFFFFFFFFFFFFFFFFFFFFFFFFF90
:10008000FFFFFFFFFFFFFFFFFFFFFFFFCFEFCDBF32
:10009000D0E1DEBFC0E0D0E100E202B900E011270C
:1000A0000093610008871987EC2FFD2F05E310E00E
:1000B0001293029307E00293CE2FDF2F60D3EC2F31
:1000C000FD2F08EE13E01293029304E6112712931A
:1000D0000293CE2FDF2F8ED349D4EC2FFD2FA0E239
:1000E000B1E00F9300E50D9302E70D9309E60D9340
:1000F00000E70D9302E70D9301E60D9306E70D93DC
:1001000005E60D930EE60D930FE60D9300E00D93BB
:100110000F91A0E2B1E00A2E1B2E12920292CE2F76
:10012000DF2F65D405E00EBDEC2FFD2F07E0029315
:10013000CE2FDF2F9AD400E00A8700904D001124C3
:1001400008E0202C312C002B21F0220C331C0A95C6
:10015000FACF00904C001124022813280886198633
:1001600044EF51E0002D112DE7D20C2C1D2C00E0A6
:1001700011270016110609F401C03CC000902300AD
:1001800000E2002205E0002B19F006940A95FBCF4F
:1001900001E0202E201800E0201609F401C006C05E
:1001A000009023000FED002203B805C0009023004B
:1001B00000E2002A03B8EC2FFD2F00E0029301E0DB
:1001C0000293CE2FDF2F89D4EC2FFD2F08841984C2
:1001D000129202920C2F1D2F12930293CE2FDF2F1B
:1001E00092D4EC2FFD2F0C2F1D2F12930293CE2FA4
:1001F000DF2FFDD30884198444E15527002D112DEC
:100200009BD20C2C1D2C00E011270016110609F4BE
:1002100001C05DC10A8400E0001609F401C03EC1BE
:100220000090210000E4202C202206E0002B19F091
:1002300026940A95FBCF00E0201609F401C02DC1D9
:10024000EED4EC2FFD2FA0E2B1E00F9304E50D9367
:1002500001E30D930AE30D9300E20D930EE40D9379
:1002600001E60D9300E70D9305E60D9304E70D936A
:1002700009E60D9300E00D930F91A0E2B1E00A2E84
:100280001B2E12920292CE2FDF2FB1D30AE21EE371
:100290002FEF2A95F1F71A95D9F70A95C1F70000C3
:1002A0000000EC2FFD2F07E00293CE2FDF2FDDD3D0
:1002B0000E821F82EC2FFD2F00E0029301E00293DB
:1002C000CE2FDF2F0AD4EC2FFD2F0E801F8044E6A7
:1002D0005527002D112D30D2002E112E02920C2FF9
:1002E0001D2F12930293CE2FDF2FA1D4EC2FFD2FC1
:1002F0000C2F1D2F12930293CE2FDF2F78D3EC2FCC
:10030000FD2F0EE20293CE2FDF2FEDD4EC2FFD2F29
:100310000E801F8044E65527002D112D0DD20C2C88
:100320001D2C02920C2F1D2F12930293CE2FDF2F24
:100330007ED4EC2FFD2F0C2F1D2F12930293CE2F66
:10034000DF2F55D3EC2FFD2FA0E2B1E00F9306E590
:100350000D9300E20D9300E00D930F91A0E2B1E048
:100360000A2E1B2E12920292CE2FDF2F40D34E80E8
:100370005F8000EE11E022244016510608F420941C
:1003800008E012E000240415150508F40094022882
:10039000002809F001C029C0EC2FFD2FA0E2B1E038
:1003A0000F9303E40D9308E60D9309E70D9302E61E
:1003B0000D9301E60D9300E00D930F91A0E2B1E0E3
:1003C0000A2E1B2E12920292CE2FDF2F10D3EC2F6B
:1003D000FD2F00ED17E0129302930CE211E012934F
:1003E0000293CE2FDF2F06D219C0EC2FFD2FA0E2F3
:1003F000B1E00F930FE40D930BE60D9300E20D9324
:100400000D930D9300E00D930F91A0E2B1E00A2E41
:100410001B2E12920292CE2FDF2FE9D20A8401E026
:10042000000E0A8604E51EE32FEF2A95F1F71A95D0
:10043000D9F70A95C1F7000001E00A95F1F7EFD36B
:10044000EC2FFD2FA0E2B1E00F9304E50D9302E342
:100450000D930AE30D9300E20D930BE40D930FE669
:100460000D930DE60D9305E70D930EE60D9309E64A
:100470000D930BE60D9301E60D9303E60D9305E650
:100480000D9300E00D930F91A0E2B1E00A2E1B2E18
:1004900012920292CE2FDF2FAAD219C00A8401E055
:1004A000001609F401C013C00090210000E4202CC4
:1004B000202206E0002B19F026940A95FBCF01E0DC
:1004C000201609F401C002C000E00A8700C035CE42
:1004D000FFCF00903B0004E0002A0BBA000001E0CF
:1004E0000A95F1F700903B000BEF00220BBA08953C
:1004F000229700EA1FE0088319830880198022965A
:10050000EC2FFD2F0895022D003079F115E1000048
:1005100000000000000000000000000000000000DB
:10052000000000000000000022EC000000000000BD
:1005300000000000000000000000000000000000BB
:10054000000000002A9500000000000000000000EC
:10055000000000000000000000000000000000009B
:1005600089F71A9509F70A9589F6012D003079F176
:1005700013E0000000000000000000000000000088
:1005800000000000000000000000000024E0000067
:10059000000000000000000000000000000000005B
:1005A00000000000000000002A950000000000008C
:1005B000000000000000000000000000000000003B
:1005C0000000000089F71A9509F70A9589F6002DB1
:1005D0000695069519F000000A95E9F70895442458
:1005E00055246624771880E220F4400E511E621EC6
:1005F000731E40FD401A40FD510A40FD620A40FD55
:10060000730A7594679457944794779567955795AF
:1006100047958A9549F70895B32EB72637FF08C046
:1006200030952095109500950F5F1F4F2F4F3F4F2E
:1006300057FF08C070956095509540954F5F5F4F8C
:100640006F4F7F4FCC24DD24EE24FF1881E2001F82
:10065000111F221F331F8A9559F4B7FE08C0309529
:100660002095109500950F5F1F4F2F4F3F4F089516
:10067000CC1CDD1CEE1CFF1CC41AD50AE60AF70AC6
:1006800030F4C40ED51EE61EF71E8894E0CF089401
:10069000DECF089500903B000FE0102C1022088060
:1006A00000EF002201280BBA14DF00903B000FE09E
:1006B000202C2022188004E0012C002B19F0000CC3
:1006C0000A95FBCF02280BBA04DF188002E001155F
:1006D00008F401C005C0000005E30A95F1F70BC05E
:1006E0000FE115E020E12A95F1F71A95D9F70A955F
:1006F000C1F7000000002196EC2FFD2F08952297EE
:1007000000E00983298033240A801B80020C131C1B
:10071000A02DB12D2C9000E0201609F001C005C0DD
:10072000098001E0000E0982EDCF0980088208806F
:100730002496EC2FFD2F0895CC24DD1881E1001FB5
:10074000111F8A9509F40895CC1CDD1CC41AD50A22
:1007500020F4C40ED51E8894F2CF0894F0CF0895EB
:10076000CC1889E0001F8A9509F40895CC1CC41A9E
:1007700018F4C40E8894F6CF0894F4CF0895209707
:1007800009801A8000922F011092300101E0088048
:10079000402E002819F0440C0A94FBCF40923101FE
:1007A000042C00940092320109801A8001E0112784
:1007B000202C201A312C310AA22DB32D0C900428A4
:1007C000A22DB32D0C9200902F011090300102E069
:1007D0001127402C401A512C510AA42DB52D2C90D4
:1007E000009032010220A42DB52D0C922396EC2FFF
:1007F000FD2F08952E977CDE08EE13E02227332785
:1008000022243324402D512D622D732DE8DE042E39
:10081000152E262E372E0889198922273327402F97
:10082000512F622F732F002D112D222D332DF4DE29
:10083000002E112E222E332E088219822A823B820C
:10084000088019802A803B80889437FC089437946C
:10085000279417940794088219822A823B824E8536
:100860005F85662777270889198922273327B7DE0E
:10087000042E152E262E372E08EE13E022273327BE
:10088000402F512F622F732F002D112D222D332D2C
:10089000C3DE002E112E222E332E088619862A86BC
:1008A0003B8640902F015090300102E01127042C2C
:1008B000001A152C110A0C861D8601E0112722272B
:1008C00033270C831D832E833F8301E011272227CA
:1008D0003327488459846A847B8440165106620613
:1008E00073060CF001C03EC0AC85BD854C900090F5
:1008F00031010428A0912F01B09130010C920880A1
:1009000019802A8000DEAC85BD854C9000903201B4
:100910000420A0912F01B09130010C920880198021
:100920002A80F1DD8C809D80AE80BF804884598410
:100930006A847B8484149504A604B70409F001C07A
:1009400011C00C801D802E803F8001E011272227DE
:100950003327000E111E221E331E0C821D822E8292
:100960003F82B3CF6296EC2FFD2F08950FEF0ABBA5
:1009700007E514E220E12A95F1F71A95D9F70A95CF
:10098000C1F7000002E00A95F1F700903B000FE08C
:10099000002200E2002A0BBA9CDD06E01DE020E107
:1009A0002A95F1F71A95D9F70A95C1F7000001E0E9
:1009B0000A95F1F7EC2FFD2F08E20293CE2FDF2FDF
:1009C00069DEEC2FFD2F01E00293CE2FDF2F62DED8
:1009D000EC2FFD2F06E00293CE2FDF2F5BDEEC2FF6
:1009E000FD2F0CE00293CE2FDF2F54DE08952297C7
:1009F00000903B0001E0002A0BBA00E00883EC2FD6
:100A0000FD2F0A801B8012920292CE2FDF2F77DEFD
:100A100011E0002D011B0983298000E0201608F059
:100A200001C01AC0EC2FFD2F288033240A801B80C0
:100A3000020C131CA02DB12D0C900292CE2FDF2F93
:100A400029DE49802880241409F001C005C00880EF
:100A500001E0000E0882E0CF00903B000EEF002284
:100A60000BBA2496EC2FFD2F0895229700E40A80FC
:100A7000002A07B807EC06B90090260000E4202CF5
:100A8000202206E0002B19F026940A95FBCF00E007
:100A9000201609F401C002C00000EECF009024002F
:100AA00011240882198200902500112408E0202CCE
:100AB000312C002B21F0220C331C0A95FACF088030
:100AC0001980022813280882198207E806B90880CD
:100AD00019802396EC2FFD2F0895EC2FFD2F088011
:100AE00006E0102C002B19F0110C0A95FBCF0980A1
:100AF000010C00E8002A0292CE2FDF2FCBDD2296D8
:100B0000EC2FFD2F0895239701E008832D803E8070
:100B100009E011270215130508F401C004C008807C
:100B200001E0000E08822D803E8003E611270215A9
:100B3000130508F401C004C0088001E0000E08821B
:100B40002D803E8007EE13E00215130508F401C066
:100B500004C0088001E0000E08822D803E800FE076
:100B600017E20215130508F401C004C0088001E073
:100B7000000E08820B801C80A02DB12D0F9300E287
:100B80000D930D930D930D930D9300E00D930F9125
:100B9000288000E0021508F401C033C00D801E80DB
:100BA0004AE05527002D112DC7DD0C2C1D2C098284
:100BB0001A8249805A802D803E80022C0418132C02
:100BC00015084AE05527002D112DB6DD002E112EF7
:100BD0000D821E82288001E0022C001A202C332472
:100BE0000B801C80200C311C09801A8000E3000E51
:100BF000A22DB32D0C92288001E0022C001A08824D
:100C0000C7CF0B801C8005E010E0000E111EA02D48
:100C1000B12D00E00C932796EC2FFD2F0895EC2FBB
:100C2000FD2F01E00293CE2FDF2F34DD08952297B0
:100C300001E008832C8009E0021508F401C004C01B
:100C4000088001E0000E08822C8003E6021508F4FB
:100C500001C004C0088001E0000E08820A801B80E9
:100C6000A02DB12D0F9300E20D930D930D9300E095
:100C70000D930F91288000E0021508F401C025C0F3
:100C80000C804AE0002D6CDD0C2C098249802C8000
:100C9000022C04184AE0002D63DD002E0C8228800F
:100CA00001E0022C001A202C33240A801B80200C27
:100CB000311C098000E3000EA22DB32D0C92288078
:100CC00001E0022C001A0882D5CF0A801B8003E0C5
:100CD00010E0000E111EA02DB12D00E00C93259602
:100CE000EC2FFD2F089500903B0001E0002A0BBA85
:100CF000EC2FFD2F08800292CE2FDF2FCBDC00904F
:100D00003B000EEF00220BBA2196EC2FFD2F089529
:00000001FF
